:030000000219FDE5
:03000B000200AA46
:03002B0002015679
:03005B000202E8B6
:030073000202D5B1
:1000800002030406080C10182030406080040608A3
:100090000C10182030406080A0C00003070F1F0D17
:1000A0000D04050D050205030302C2AFC0D0C0E078
:1000B000206214E5256009E473E525F4F58AD2622F
:1000C000D0E0D0D0D2AF3285268AC262E526F46075
:1000D00029D0E0D0D0C293C297C295D2AF32C2939A
:1000E000C297C295206F0C206609740ED5E0FDE51D
:1000F0007B4290D0E0D0D0D2AF32758A00C28DD290
:100100006201F301B9306805206602D29301B9306B
:100110006805206602D29701B9306805206602D2D0
:100120009501B9C29230680A206607740CD5E0FDCB
:10013000D29301B9C29630680A206607740CD5E0E4
:10014000FDD29701B9C29430680A206607740CD5B5
:10015000E0FDD29501B9C2AFC2AD53E6EFC0D0C049
:10016000E0D2D3D2AFC2CEE52A6007207449152A67
:1001700021B77800790020742EE580307E01F430BC
:10018000E50278FF53DACF207E0343DA20307E0386
:1001900043DA10C2D8C271E580307E01F430E50246
:1001A00079FFC3E89970CB306103752A1820740376
:1001B000752A18885CD27020740DE52B6004152B0D
:1001C00021C743DA01C2D82070024136A85C206101
:1001D00002C2702074367982B70431C3E894F040CB
:1001E0000374F0F8E8C4540F28F87984B703024187
:1001F0000CC313C3138721200802C313200A06C3AC
:10020000C898F8410C28F8500374FFF88822E52DAF
:1002100054066022206B1FE536C333C333F8E56410
:10022000C313C313F9C3952240028922E82522F59E
:100230002250037522FF7882B6044E852224A8241A
:10024000C3E52495614002A861C3E895634002A814
:10025000638825E56670024187C3E8AA669A500361
:10026000E8FAE4F9EAC333FBE568F45B29400D25BD
:1002700067F8E56760021567400B41870AC3E567C9
:100280009A5002056778FF8826C3E525944040020E
:10029000D26420CF0AD0E0D0D043E610D2AD32C233
:1002A000CF053A7801E52A6005307402152AC3E5C6
:1002B0005C94014005755F0041CB75600075690075
:1002C000E55F2401F55F5003755FFFD0E0D0D043B8
:1002D000E610D2AD32C2AF53E67F7592FA7593FF46
:1002E000C260759104D2AF32C2AF53E6EFC2ADC067
:1002F000D0C0E0C0F0D2D3D2AFA8FBA9FCC2D830A6
:100300007102614F53DACF207E0343DA10307E034F
:1003100043DA20D271E580307E01F420E5026126C7
:1003200088278928A17C53DACF207E0343DA203046
:100330007E0343DA10C2D8C271307402A16878001B
:10034000E580307E01F430E502A168885CA150535D
:10035000DACF207E0343DA20307E0343DA10C27105
:10036000206102812853DACF207E0343DA10307EE9
:100370000343DA20C2D8D27188578958C3E895550B
:10038000F8E99556F97B007E087A00C3E8948CE979
:1003900094005005755B00811A882178A2E6A82197
:1003A0006055C3E894C8E994005008E4D2E4FB7AAD
:1003B0000A61F5C3E89468E994015008E4D2E3FBCC
:1003C0007A0F61F5C3E894D0E994025008E4D2E2D0
:1003D000FB7A1E61F5C3E894A0E994055008E4D2C5
:1003E000E1FB7A3C61F5C3E89498E994085008E48D
:1003F000D2E0FB7A787E00C3E89559FCE9955AFD76
:1004000030E70AECF42401FCEDF43400FD755B00E8
:10041000C3EC9AED9E5003755B018859895A855744
:10042000558558567802A150C3E89527F8E99528D4
:10043000F9307C02A134307B02A134307A02A12D44
:10044000207502814BE9FDE8FC816AE9C313F9E8F4
:1004500013F8307902A12DE9C313F9E813F83078C5
:1004600002A12DE9C313FDE813FC20612CC3EC9419
:0F0470001CED940240028181ED701EC3EC94C814
:10047F0050180529E52970021529C3E529940A505A
:10048F0002A168755C00D270A168E5296002152988
:10049F007888E6F97400207F087896B90302789E71
:1004AF00E624FAFEE43400FFC3EC9EFCED9FFD92C0
:1004BF0008B90310A2085007207609D27681D330ED
:1004CF007602C276A2085016B9030DECF42401FC93
:1004DF00EDF43400FD0204ED78007900A134B90386
:1004EF0015EC33FCED33FDC3EC940AFCED9400FDE9
:1004FF0050047C007D00C3EC94FFED94004006781F
:10050F00FF7900A134EC8572F0A4C5F0A2F733F89F
:10051F007900400302055078FF7900020550E9C3C6
:10052F0013F9E813F8307C0EE9600278FFC3E81383
:10053F0038F8E43400F9C3E894FFE99400400278F6
:10054F00FF885CD270206102A168741FF4552F4B95
:10055F00F52FC274EB7002D274752A1830740375BC
:10056F002A0A306102A17C20740353DAFE2074033F
:10057F00752B06D0F0D0E0D0D0D2AD43E610327953
:10058F00010205AC79030205AC790A0205AC791EAC
:10059F000205AC79640205AC79C80205AC7817E4A2
:1005AF00D5E0FDD8FAD9F6227A147B780205D37AF2
:1005BF00107B8C0205D37A0D7BB40205D37A0B7BAB
:1005CF00C80205D37902E4C296D5E0FDD297D5E0F3
:1005DF00FDC297D5E0FDD296D5E0FDE920E002D22D
:1005EF009330E002D295E573D5E0FDE920E002C239
:1005FF009330E002C2957496D5E0FDD9C9EAF8D5DB
:10060F00E0FDD8FBDBBEC29622C37C007D0075F0F7
:10061F000005F0EA33FAEB33FB50F6EB13FBEA136A
:10062F00FAC3E9FFE8FEE89AF8E99BF95004EFF9FD
:10063F00EEF8B3EC33FCED33FDD5F0DFEDF9ECF86C
:10064F0022E889F08A20D2D4F8A9F07B0030F70B8A
:10065F007BFFF42401F8E9F43400F9E88520F0A4D5
:10066F00ADF0F8E98520F0A4AFF0FEED2EF974009F
:10067F003FFA7C04C3EA13FAE913F9E813F8DCF440
:10068F008BF030F70AE8F42401F8E9F43400F9E8C4
:10069F0089F0C2D4F8A9F0227882B60403020702C7
:1006AF00C3E55C940140030206CC852224E4F544A3
:1006BF00F545F546F547F548C26E0207027882E622
:1006CF00FCD26EE522F523783879C7AA40AB41C337
:1006DF00EB13FBEA13FAEC146013C3EB13FBEA13EF
:1006EF00FAEC14146007C3EB13FBEA13FAD1188862
:1006FF0044894522C3E5449523F8E5459400F95014
:10070F000CC3E89480E994FF4016020733C3E894C2
:10071F007FE994005003020733787F790002073393
:10072F00788079FF8849894A22E5492546F8E54AC4
:10073F003547F9854A20E4300701F43548FA30E7A8
:10074F0009C3EA94F04015020771C3EA940F5003EE
:10075F0002077178FF79FF7A0F020771780079002D
:10076F007AF0C3E5249561500AC374019524500BA8
:10077F0002078FE54A20E70E02078FE54A30E706AA
:10078F00884689478A482278A5E6FAC3E54933F8AF
:10079F00E54A33F9D150E930E70BC3E89480E99487
:1007AF00FF4013E1C9C3E8947FE994005002E1C907
:1007BF00787F7900E1C9788079FFE820E715C3E5F4
:1007CF002398F84009C3E8940140030207F0780129
:1007DF000207F0E8F424012523F840030207F0781C
:1007EF00FF884B2278A6E6FAA847A948D150E930EE
:1007FF00E70CC3E89401E994FF4016020824C3E80C
:10080F0094FFE99400500302082478FF790002084E
:10081F0024780179FFE920E715C3E54B98F84009E3
:10082F00C3E89401400302084B780102084BE8F437
:10083F002401254BF8400302084B78FF88242278C7
:10084F00FFC26420693D206A12D264C3E541940A55
:10085F004009C3E52594405002C26479A1E76023A3
:0D086F00E541601F74FF8541F0848539F07C
:10087C00306A0375F005A4F8C5F0600278FFC3E890
:10088C0095645002A864886322C3E5409440E54116
:10089C009401E56350031401A6046002F56322027F
:1008AC0008AE2275E890227883E6FFE5E820ECF7A5
:1008BC00A8BDA9BE0570C3E57094084052757000C0
:1008CC00E9FA79A0E76044EA7007E571601B020859
:1008DC00E9C3E895716010E5715006600C140208CC
:1008EC00F50460F90208F5E571F571C3946D401BD0
:1008FC007561C0C394044013756180C39404400BAC
:10090C00756140C39404400375610075BB0822E512
:10091C00612410500274FFF5617982B70402214200
:10092C00C3A861E524985002A824C3E8956340024B
:10093C00A86388258826E570B4070375BB1022745C
:10094C003279A787F0A4C5F0A2F733F8C3E8956114
:10095C004002A8618822882488258826886422750C
:10096C0040007541F022C2AF75C820A8CCA9CDAA11
:10097C003A30CF010A75C824D2AFAB3BAC3C883BB4
:10098C00893CC3E89BF8E99C206908F9306702416F
:10099C007E21DBAD3D8A3DF9EA9DFA600478FF7952
:1009AC00FFAE3EAF3F8B3E8C3FA83BA93CC3E89EBD
:1009BC00F8E99FF9C3E54113FBE54013FAE82AF582
:1009CC0040E93BF54150067540FF7541FF4125AAB2
:1009DC0040AB41AC40AD417E047F02C3EB9404407C
:1009EC00021E1FC3EB940840021E1FC3ED13FDEC47
:1009FC0013FCDEF7C3EA9CFAEB9DFBEF6009C3E93D
:100A0C0013F9E813F8DFF7EA28FAEB39FB8A408B85
:100A1C004150067BFF8B408B41C3EB94025002D2BA
:100A2C00673069047F0341507892E6FFC3E5379441
:100A3C008240110FC3E53794A040010FC3EF940619
:100A4C0040027F057E02E541C4540FF9E541C454D0
:100A5C00F0F8E540C4540F28F8C3E89EFAE9940076
:100A6C00FB4009C3EA9402EB940050047A02E4FBC5
:100A7C0041CAAA40AB41EBC4FEEAC4540F4EFCC3BE
:100A8C00EA9CFAEB9400FBC3E813C313F8EA28FAC8
:100A9C00EB3400FB8A408B41C3EB94024002C267EB
:100AAC007802EBC4FE7B00EAC4540F4EFAC3EA98FA
:100ABC00FA4005C3940250027A027892E6FF306045
:100ACC000241CA855192855293D26043E680C3E4B9
:100ADC009AF8E49BF93067026156E8FAE9FBD3E92E
:100AEC0013FDE813FC88518952C3EF94036038EF6F
:100AFC0020E00DE82CF8E93DF9ECFAEDFB020B1FB8
:100B0C00E828F8E939F9C3E82402F8E93400F97A5D
:100B1C00FE7BFFC3EF9403400E8A538B54884D89A0
:100B2C004E8C4F8D50618A885389548A4D8B4E8CD4
:100B3C004F8D503069127553F07554FF754FF07529
:100B4C0050FF7551F07552FF618AE8FAD3E813FC37
:100B5C008851C3EF94036020EF20E007E82CF8ECF9
:100B6C00FA6176E8282402F87AFEC3EF9403400871
:100B7C008A53884D8C4F618A88538A4D8C4FE56817
:100B8C00C3335002646BF5683060026194753402B3
:100B9C00D26043E680E52D54066034A840A941C3D9
:100BAC00E913F9E813F8C3E913F9E813F830690409
:100BBC00E92440F9C2AF53E67F759100C3E498F580
:100BCC0094E499F595759104D26043E680D2AF22F6
:100BDC00D265754300752000306C03752040020B04
:100BEC00FBD265754300752040306C03752000788E
:100BFC00017901206720E52D54066002C265791445
:100C0C00E541C313700104F8C39414400278143006
:100C1C006904781B791B206010E543600C30690374
:100C2C00D53404D26D819D719C0543E59B5440B530
:100C3C002002818730690908C3E899400118812294
:100C4C0020650A08C3E899400261FB8122C265C293
:100C5C00AF53E67F7591003067127594007595FE61
:0E0C6C00759104D26043E680D2AF61FBAE40CA
:100C7A00AF41C3E49EF594E49FF595816CC3E533D7
:100C8A009401500261FB30650261FBD802819B81AD
:100C9A0022C26DC2AF53E67F759100855394855485
:100CAA0095759104854D92854E93D26043E680D224
:100CBA00AFE52D54066008206A020533020CD930CC
:100CCA006D0D206C0A2065071581158102155C22BD
:100CDA0078003064053065027801E53775F007A4BD
:100CEA00F9E5F028F5F0E9A2F013A2F113A2F21344
:100CFA00F537C394785003753778C3E5379538408C
:100D0A0008D266C293C297C295306002A113854F7A
:100D1A0092855093D26043E68022207D16C2AF7539
:100D2A004202C296D292306202D295D2AF759F1118
:100D3A00020F13C2AF754202C296D294306202D237
:100D4A0093D2AF759F11020F13307243207D20C2D8
:100D5A00AF754203900134757B40C295C2943062EC
:100D6A0004D297A171D296D2AF759F10020F13C207
:100D7A00AF754203900134757B40C293C2923062D0
:100D8A0004D297A191D296D2AF759F13020F132066
:100D9A007D17C2AF75420390010FC295306202D22D
:100DAA0097D2AF759F10020F13C2AF75420390011D
:100DBA000FC293306202D297D2AF759F13020F13FC
:100DCA00207D16C2AF754204C292D294306202D21A
:100DDA0097D2AF759F13020F13C2AF754204C29424
:100DEA00D292306202D297D2AF759F10020F13309F
:100DFA007243207D20C2AF754205900123757B04A2
:100E0A00C297C296306204D293C117D292D2AF75FA
:100E1A009F11020F13C2AF754205900145757B10F1
:100E2A00C297C296306204D295C137D294D2AF75B6
:100E3A009F11020F13207D17C2AF7542059001055D
:100E4A00C297306202D293D2AF759F11020F13C2BA
:100E5A00AF754205900119C2973062EBD295D2AFB5
:100E6A00759F11020F13207D16C2AF754206C294F8
:100E7A00D296306202D293D2AF759F10020F13C27C
:100E8A00AF754206C292D296306202D295D2AF753F
:100E9A009F13020F13307243207D20C2AF754201A7
:100EAA00900145757B10C293C292306204D295C1FB
:100EBA00BDD294D2AF759F13020F13C2AF75420110
:100ECA00900123757B04C295C294306204D293C107
:100EDA00DDD292D2AF759F10020F13207D17C2AFD9
:100EEA00754201900119C293306202D295D2AF7550
:100EFA009F13020F13C2AF754201900105C29530CC
:100F0A006202D293D2AF759F10C266229001037516
:100F1A007B00C293C297C295C292C296C294C26221
:100F2A0022788076090876090876040876FF08761A
:100F3A00030876FF08760808760108760108760124
:100F4A00788C76010876FF0876FF0876FF0876FF28
:100F5A000876FF0876030876FF0876FF0876FF080A
:100F6A0076250876D008762808765008760408761A
:100F7A00FF08760208760008767A0876FF08760176
:100F8A00087601087600087603087600227887E654
:100F9A00FFC2727888E6C394036008C27DE630E136
:100FAA0002D27DC27E7889E630E102D27EC3EF9416
:100FBA00026008758E01D273020FCA758E00C27361
:100FCA00227880E6149000809378A5F67881E6145A
:100FDA009000809378A6F67886E61490008D937830
:100FEA00A7F67886E6F539C3940250037539027874
:100FFA009CE67538FFB402037538A0B4030375384C
:10100A008278A3E61490009A93F566120F162222AC
:10101A007896E6FA7897E6FB7888E6B40305C3EB98
:10102A00940EFB307F047A007BFFC3EB9AFCC394D7
:10103A008250027C827572000572EC8572F0A4C33C
:10104A00E5F0947D40F222D27F111A12059D7A00B2
:10105A007B007C10120593E55C2AFA74003BFBDCEA
:0F106A00F37C04C3EB13FBEA13FADCF7FEC27F3F
:10107900111A22E5EF20E6037520000520903FFFB5
:10108900E520146006901DFF146000930460037549
:10109900EF1253D9BF7581C043FF8012058E75EFDA
:1010A9000243B203E5B3240220E70DF521E5E3206D
:1010B900E0068521B343E301120F167580FF75A47D
:1010C9000075F1B275D4DF75900375A5FC75F2FC56
:1010D90075D50375A60175E241120F16E4F8F6D825
:1010E900FD756801120F2B1215AD7898867375304E
:1010F90001C2AF1205A71205B712059D1205BE124E
:10110900059D1205C512059DC2AF78FA79FA308599
:1011190007D9FBD8F7021C00120F97120FCB111930
:10112900111A78988673120F1675881075890275C9
:10113900C82475910475D84075A82275B80275E65A
:1011490090759B80759D0075D10E75BC5875BB084F
:1011590075BA1175E88012058ED2AF1208AB7536D3
:101169000053DACF207E0343DA20307E0343DA10BE
:1011790043DA01C2D8C2711205A7D2617B037A0C86
:10118900E55B70077A0CDB0302111112059D2070D3
:1011990003021111C270E55CC3940240E1E52F54CA
:1011A9001F855E5DF55EB55DD5DAD5C26153DACFCF
:1011B900207E0343DA20307E0343DA10C2D8C2719D
:1011C90078A2E67008D274E52F54E0F52FC2757540
:1011D90029001205A2307409C3E529940A4002D2F4
:1011E9007512059378023074027800C3E55C984063
:1011F900F0C2AF1205B71205B71205B7D2AF120583
:10120900A7754C007888E6B4030241E91205937882
:101219008CE6C3940150030212E9E530C3940150EE
:10122900030212E9207435C3E55C94FF50030212EE
:10123900E9C2AF1205CCD2AF1205A2C3E55C940195
:1012490050EFC2AF1205B71205981205B7D2AF1207
:1012590005A2C3E55C94FF40E90217557F02D27FDE
:10126900111A1205A2C2AFC27F111AAE5CC3E55CA6
:10127900947FD2AF407412058EC2AF1205CCD2AFA3
:10128900DFDC1151C3EE7897F61205A71215EF129C
:1012990016D87F0AD27F111A1205A2C2AFC27F11D6
:1012A9001AAE5CC3E55C947FD2AF50E612058EC2DC
:1012B900AF1205B71205981205B7D2AFDFD6115193
:1012C900EE24037896F61205A71215EF12170712E6
:1012D90005A2111AC3E55C94FF5002412D0217556E
:1012E900C3E55C954C4003855C4C1205A2780179F5
:1012F90088E7B403027805C3E55C984002410DC252
:10130900AF1205CC1205CC1205CCD2AF1205A775C8
:101319003000E4F531F5320531E531F4703F05323D
:10132900789AE67819146012783214600D787D1471
:10133900600878FA146003753200C3E53298401DDD
:10134900120F1612058E153275310078998673C2FF
:10135900AF1205CCD2AF789886731205A212059800
:10136900E52A70053074022111780120740278068B
:10137900C3E55C9840A17888E6C39403600312052D
:10138900A2E52A7003021111C2AF120F16E4F52269
:10139900F523F524F525F526F567D2AF7885E6C35B
:1013A90033F565E4F544F545F546F547F548F57037
:1013B900F52CF52DF53775700875BB1012058E12D1
:1013C90008AFE5E820ECFBA8BDA9BEE97001F888E3
:1013D900711208B375700875BB10120F97C2AF75FB
:1013E90061FF12094B852261852262852263D2AF92
:1013F90075220175240175250175260185606975B8
:101409006A017888E6B40307C27D307602D27DD2BC
:1014190068D269753300120E70120E9F12096B1291
:10142900097212096B12097212096B120BED12067D
:10143900A7120CDA120D24120972120BDC306E039A
:1014490012070320670312084E306703120895122A
:101459000CDA120D53120972120BED306E031207DA
:0D14690038120CDA120DCA120972120BDCD7
:10147600306E03120796120CDA120DF91209721267
:101486000BED306E031207F3120CDA120E7012090E
:10149600721208AF120BDC120CDA120E9F1208B38E
:1014A6001209723069328564618564628560697586
:1014B6006A0179187A0CC3E53399400FC269D26A7A
:1014C6008A358564618564630214DEC3E55C940134
:1014D6004003021434021564306A1D206C1AE53587
:1014E600147006C26AD26B8134F535C3E55C94018B
:1014F600400302143402156475360078FA79A4E7BD
:1015060060027803C3E55F985054307404E52A609E
:101516004D7888E6B40317207D05207607A1343080
:101526007602A134206C07D26C856461817378F0F1
:10153600306C058564617820C3E54198500281349A
:10154600306C1BC26CC27D307602D27DD26A753594
:101556001285646181340536E55C6002A1677536E3
:1015660000C2AF120F167887E6FE7602120F977842
:1015760087EEF6E4F522F523F524F525F526F5653F
:10158600752C00752D00D2AF1205A2120F1678A485
:10159600E66006D293D297D295307409C3E53694A5
:1015A6000440022111611B901A0D7820121631E5B4
:1015B60020B4550CA3121631E520B4AA030215CFA8
:1015C600120F2B1215EF0215EE901A0378807B0A84
:1015D600121631A308DBF9901A0F788C7B191216B4
:1015E60031A308DBF9901A2822C2AF121670121620
:1015F6004A901A00740E121636A37406121636A3F3
:101606007415121636901A0378807B0A121635A3C3
:1016160008DBF9901A0F788C7B19121635A308DBB4
:10162600F9121683121661901A2822E493F622E61E
:10163600438F01538FFD75EF0275B7A575B7F1F0AE
:10164600538FFE22438F02438F0175EF0275B7A5B4
:1016560075B7F1901A0DF0538FFC22901A0D745540
:10166600D136901A0E74AAD136227A3079D07820E3
:10167600901A40D131E520F709A3DAF7227A3079BA
:10168600D0901A40E7D13609A3DAF922AB74A875CF
:10169600BB01027980BB02027981BB03027982BB5E
:1016A60004027984BB05027986BB06027992BB07E0
:1016B600027987BB080279A3BB0902799CBB0A029F
:1016C6007988BB0B027989E8F7227C051205A7DC2D
:1016D600FB22C2AF1205B71205BE1205C51205CC14
:1016E6001205981205B71205BE1205C51205CC12D1
:1016F60005981205B71205BE1205C51205CCD2AF64
:1017060022C2AF1205CC1205C51205BE1205B712CC
:1017160005981205CC1205C51205BE1205B71205AD
:10172600981205CC1205C51205BE1205B7D2AF2216
:10173600AE74AF75C2AF1205B71205B71205B71270
:101746000598DEF21205CC120598DFF8D2AF22D149
:10175600D8D1D0D1D0757401757501757600F13682
:101766007C05AD5C1205A7C3ED955C70F5C3E55C21
:101776009401400AC3E55C94FF4032021791D1926E
:10178600B1EFD1D8C2AF75EF12D1D0DCD50576C393
:10179600E5769403500280C6D1D00575E5741490A1
:1017A600009F93F808C3E57598500280AED1D0D15A
:1017B600D00574C3E574940C5002809C120F2BB1B3
:0817C600EFC2AF75EF12D1D0A4
:0319FD0002107C59
:101A00000E0615090904FF03FF0801010155AA018B
:101A1000FFFFFFFFFF03FFFFFF25D0285004FF0259
:091A2000007AFF0101000300FF40
:101A4000235475726E696779383041232020202035
:101A500023424C48454C4923463333302320202031
:101A60002020202020202020202020202020202076
:101C0000C2AFC2D353D9BF7581C043B20343FF8073
:101C1000752438752503B1C975EF0275E24043F1AB
:101C20002053A4DF75D4FFD2857DFA780379E67C52
:101C300010752200752300901DD67B0675249875BB
:101C400025013085028142208508D8FBD9F9DCF7CF
:101C500081B4308508D8FBD9F9DCF781B4B189E4C7
:101C600093A3C39A6004DDC381B4DBDBB17B600264
:101C7000812B7B08E493FAA3B15CDBF87A30B15C8A
:101C8000752200752300B17BEAFCEBFDC3ED94FEE9
:101C9000400EB17B8A278B28ED30E0048A828B834B
:101CA000B17B7AC270D8C3ED94FE601350CEBD00F4
:101CB00025EC60097520007521FF0200008100A855
:101CC00027A9280809D804D90281D3B17FEA89AAB3
:101CD000F281C50D81A0C3ED94035049EDA2E092BD
:101CE000007AC5C3E5829400E583941C50902000DF
:101CF00010438F02438F0175B7A575B7F1F030001F
:101D00001FA827A9280809438F01538FFDD804D99C
:101D100002A12089AAE275B7A575B7F1F0A3A10DBC
:101D2000538FFC817C7AC1BD030CE493A3FAB140CC
:101D3000DCF8B138817C817EAA22AB23B15CEBFA5E
:101D4000EA6222752608C3E52313F523E52213F57D
:101D50002250066323A0632201D526EAB1C9B1C986
:101D600075260AEAF4200102D285300102C285B14B
:101D7000C9C3134002C201D526EB22B17FEAFB2082
:101D80008502A17F308502A184752608AE24AF2587
:101D9000C3EF13FFEE13FEB1CDB1C9C3EA13308513
:101DA000024480FA30E703632201C3E52313F523DD
:101DB000E52213F52250066323A0632201D526D91C
:101DC000E52265236523F52222AE24AF250E0FDE22
:101DD000FEDFFCD20122424C48656C693437316326
:041DE000F3300601D5
:00000001FF
